:1000000012C02BC02AC029C028C027C026C025C0C6
:1000100024C023C022C021C020C01FC01EC01DC0DC
:100020001CC01BC01AC011241FBECFE5D4E0DEBF28
:10003000CDBF10E0A0E6B0E0E2E9F0E002C005903C
:100040000D92A036B107D9F710E0A0E6B0E001C0EC
:100050001D92A036B107E1F70EC0D2CF9C01E0EFB0
:10006000F0E005C0CF010197F1F721503040211594
:100070003105C1F70895CFE5D4E0DEBFCDBFA59A25
:10008000AD9884EF91E0EADFAD9A84EF91E0E6DF8E
:02009000F7CFA8
:00000001FF
